:020000040000FA
:060000008316031315280E
:08000800B8000308BA00040867
:10001000B9000A08BB00CE203B088A0039088400DA
:100020003A088300B80E380E090002309F002F30C6
:100030008500D7308100C03086000F3087008312E2
:10004000031380309F00FF3085008600870020303A
:1000500084008001840A3C300402031D29280830F2
:10006000A9000030A800F030A400861B061FA014D1
:10007000B0308100A0308B00A0189C282A08A10075
:100080002018A1032D082102031851282014051659
:100090003030A40407194F28F030A4003E289921DD
:1000A0003E28201005123208310203186728071C69
:1000B0007528FF3A013EA100CF302404FF3AFC30FE
:1000C000031DFE30210503197528A5217728871CFB
:1000D0007528A100CF302404FF3AFC30031DFE3008
:1000E0002105031975289F2177283030A404300892
:1000F0002F0203188B28071D9928FF3A013EA10003
:100100003F302404FF3AFC30031DFE302105031963
:10011000992899213E28871D9928A1003F30240461
:10012000FF3AFC30031DFE30210503199928932165
:100130003E28C030A4043E28861B061F9C28861B30
:10014000B428071CA7283230B300A5219F28F0301F
:10015000A404861BB428871CB1283130B3009F212A
:10016000A928F030A4049F28F030A404061BCB2853
:10017000871DBE282F30B3009321B628F030A40489
:10018000061BCB28071DC8283030B3009921C02892
:10019000F030A404B628F030A4049F280B1D0800FA
:1001A000B03081000B11D621B621B708031DB7036B
:1001B000792124083F38FF3A031DE3288717000000
:1001C00000000717FC28B408031DF428A41BED2821
:1001D0000717000000008713F828241BF42887174E
:1001E000000000000713F828871700000000071719
:1001F000B40A013034020318B4012408CF38FF3A9E
:10020000031D072987160000000007162029B508DE
:10021000031D1829A41A11290716000000008712CF
:100220001C29241A182987160000000007121C290F
:100230008716000000000716B50A013035020318C2
:10024000B501A0186C29A50803193F29A503201B97
:100250002D29061B452920173329061B3B2920176A
:10026000A508031D4629A80A0A3028020318A80178
:100270006230A50046292013F430A5004629061B4C
:1002800045292017F430A50046292013A608031994
:100290006329A603A01B5029861B6929A01756298C
:1002A000861B5F29A017A608031D6A29A90A0A3020
:1002B000290203300318A9006230A6006A29A0139E
:1002C000F430A6006A29861B6929A017F430A6001D
:1002D0006A29A013AB210800A50B0800330884008D
:1002E00000080F39A800000E0F39A9003130A50011
:1002F0000800A70A3030A300FF308600A508031DC0
:100300008629A608031D86292B30872928308400DA
:1003100027188C2923128E29840AA31200080F396A
:10032000230486000800241B97292417FC21A4130A
:100330000800A41B9D29A417FC2124130800241ADB
:10034000A3292416FC21A4120800A41AA929A41682
:10035000FC212412080003102908AA00AA0D2A086B
:10036000AA0DAA0DAA072808AA070800AD01AC012A
:100370002E08E63CAB000318C929FF3A013EAB004A
:10038000093C031CC6296430AB07CF296D30AB0094
:10039000CF29AD00633C0318CF296330AB000A308E
:1003A0002B02031C0800AB00AC0ACF298130EC21E2
:1003B000B200F3218930EC21B100F3219130EC211E
:1003C000B000F3219930EC21AF00F321A130EC21F2
:1003D000AE0080309F0008009F00F3211F151F19F9
:1003E000EF291E0808001730B6000000B60BF529EB
:1003F00000000000000008001930B700B708031D16
:04040000FE290800C9
:02400E00323F3F
:00000001FF
